:020000020000FC
:020000001FC01F
:040014007AC0CEC020
:02001A00D0C054
:100020000DC10D0A626B2373626C2D666C6F6823C1
:100030003838765F70776D32306B5F7430340D0A0C
:1000400004E00EBF0FEF0DBF03E005B900E004B9F7
:1000500008E208B90AE307B905E10BB90AEB0AB9E6
:1000600001E000937E0001E000937F0002E005BD07
:1000700002E000938100772788279927B1E0A0E06C
:10008000002719E20D931A95E9F71BD302E0C02E61
:1000900019B11570153069F0143041F0113019F0B4
:1000A00001E011E008C00CE01AE005C008E114E12D
:1000B00002C002E318E200931D0110931E0158983C
:1000C00059983FD13ED111D130D112D12ED113D177
:1000D0002CD101EF302E00E0D02E01E005BB0093C3
:1000E0006E0003E206BB00936F0002EE00937C00FB
:1000F00028D104D103D102D156D178940ED353D153
:100100000EE100932001CDD131C32FB6409186007E
:10011000509187008820A1F0BAF4609181006F7B34
:1001200060938100882471FD43C073FF41C046196C
:100130005709A42EB52E7260777F42E0C42E38C0D6
:1001400071FD36C0839434C0682D613021F4642E73
:10015000752E83942DC04F935F93461957097F9056
:100160006F90403961E0560708F1483562E0560764
:10017000E8F472FD05C040931B0150931C017460AC
:100180004091810040644093810040E8842E18999A
:1001900002C078600DC04427A42EB42E726042E0E5
:1001A000C42E409181004F7B409381008824777F4B
:1001B0002FBE18952FB67E7F2FBE18952FB670686C
:1001C000EE2009F0EA94CC2059F4189B04C044278F
:1001D000A42EB42E06C0A0901701B090180101C043
:1001E000CA9440912701442311F5409125014423ED
:1001F00029F05D984A954093250115C0409126014C
:10020000442329F05F984A95409326010CC0409101
:10021000230140932501409124014093260144E1AC
:100220004093270109C04AE04093270105C04A9541
:10023000409327015D9A5F9A2FBE18952FB676FDE1
:1002400032C0906140B745FD9F7E432D552D541718
:1002500038F44A9469F450911D01452E4A9507C01F
:1002600039F04A9429F450911E01452E4395342EBD
:10027000706475FF03C081FF5B9807C074FF03C003
:1002800081FF419802C081FF4498432D425A3AF4BD
:100290004A5F433040F047704A95F1F704C04095FB
:1002A000459546BD1EC075FF03C080FF5B9A07C021
:1002B00074FF03C080FF419A02C080FF449A432D1F
:1002C0004F93459546BD4F917F7B4D3918F4826021
:1002D0008E7F07C0413F18F08D7F816002C08D7F07
:1002E0008E7F93FD81602FBE189538EC10E509C014
:1002F00034EB14E606C030EA18E703C034E618EC25
:1003000000C0002706BD4598419A06B50032E9F7BE
:10031000459A419828E0002706BD06B50317E9F77E
:100320002A95C9F71A9569F708951FE028E0002774
:1003300006BD06B50F3FE9F72A95C9F71A95B1F73B
:10034000089510E828E0002706BD06B50F3FE9F73D
:100350002A95C9F71A95B1F7089505E800937A0030
:1003600000917B000F7B00937B0020917C0002EECC
:1003700000937C000000000005EC00937A00000070
:1003800000917A0006FDFCCF009179000F9305E003
:1003900000937A0000917B00006400937B000F9132
:1003A00020937C000895D9DF00931F019F7B073DB8
:1003B00048F40A3C50F40C3B58F40F3A60F400E067
:1003C00014E00BC004E010E008C003E011E005C039
:1003D00002E012E002C001E013E000932301109359
:1003E000240108958F7E71FF01C0797F0A2D1B2D96
:1003F00020911701309118012017310720F4009146
:1004000017011091180116950795169507952EE07E
:10041000002371F010911901109F212D10911A01E4
:10042000109F200D243608F024E62F3008F42FE02A
:10043000F22F08958F7B20910C0110910B010091F8
:100440000A01011B00930A0100910B01020B0093AA
:100450000B0100910C01004000930C012091090157
:10046000109108010091070126951795079526958B
:100470001795079520930901209308012093070100
:1004800020910A01200F20930A0120910B01211FC6
:1004900020930B0100E020910C01201F20930C0100
:1004A0000895C0E8DBEBC0931101D09312012FEF48
:1004B0003FE120930D0130930E0120930F01309303
:1004C0001001E1E0E09306013FEF309305012FEFCB
:1004D000209304010895F894000000918400109185
:1004E000850000930001109301010C0F1D1F109354
:1004F0008900009388007160789400910401109144
:100500000501E09106010093130110931401EE23FD
:1005100029F03FEF3093130130931401E6951795BE
:100520000795E695179507952091040130910501EF
:10053000E0910601201B310BE04000910001109179
:100540000101C0910201D0910301009302011093B7
:1005500003010C1B1D0B0093150110931601200FB6
:10056000311F10E0E11FEE2351F4332341F4213E0B
:1005700030F431E02CE4FF2011F40FEFF02E209343
:10058000040130930501E0930601E23008F099DFA1
:1005900000910701020F0093070100910801031F5A
:1005A00000930801009109010E1F00930901E695CF
:1005B00037952795E69537952795E69537952795AD
:1005C000E6953795279520930D0130930E012093E2
:1005D0000F01309310010895C0910D01D0910E01CB
:1005E0007ADF089570FDFECFD0911401C091130100
:1005F000F894000000918400109185000C0F1D1FDD
:100600001093890000938800716078940895C091D8
:100610000F01D0911001F894000000918400109116
:1006200085000C0F1D1F10938900009388007160D6
:10063000789484FDD7DE85FD18D086FDFBDE96FD1F
:10064000B2DE70FDFECF0895C0911101D09112016C
:1006500042DF009100010F70D01BDC3808F4DBEBA7
:10066000D093120141D040D008958F7D0F2F0D19E6
:1006700008F40EE010910601112321F410910501F8
:10068000103438F09160926019E1011760F0012F89
:100690000AC0103238F09E7F926012E3011718F002
:1006A000012F01C09C7F95FF09C02EE1021710F4B5
:1006B0000EE104C028E2021708F0022F0095502E28
:1006C0000895FEE001EF302E502E08E208B905E152
:1006D0000BB900911D01402E8160977F90620895B3
:1006E00004E00A95F1F7089576FDFECF76FFFECF80
:1006F000089508952F933F93797F71FD02C053DED3
:10070000FCCF797F71FD02C04EDEFCCF00911B0152
:1007100010911C013F912F910895ECDF202F312F74
:10072000E9DF021B130B10F4109500951123A9F7B4
:10073000007F002391F7209317013093180136951D
:1007400027953695279500E014E63327EE27339555
:10075000332309F4E395021B3F933327130B3F9197
:10076000B0F730931901E0931A010895AADFC1DFB1
:1007700039DE19DEFF30E0F30EE10095502E33270D
:1007800003E005B905E10BB90BE10A95F1F738D1A2
:100790003ED19B7F00E00093210108E2E02E81DE44
:1007A00053DF94FF10C070FD02C0946013C09CDF43
:1007B00094FDF9CF00E000932101ECD0F2D005D1F7
:1007C00011DE42DF31C070FD02C0946003C08CDFD7
:1007D00094FFF9CFDFD038DF94FD08C070FD02C070
:1007E00094600BC081DF94FFF9CF07C070FD02C099
:1007F000946003C079DF94FDF9CFD3D0F3DD24DF1B
:1008000094FF08C070FD02C094600BC06DDF94FDC2
:10081000F9CF07C070FD02C0946003C065DF94FF8C
:10082000F9CFD3D022DF10DF94FD08C070FD02C0E5
:1008300094600BC059DF94FFF9CF07C070FD02C070
:10084000946003C051DF94FDF9CFC6D0ACDDFCDE6F
:1008500094FF08C070FD02C094600BC045DF94FD9A
:10086000F9CF07C070FD02C0946003C03DDF94FF64
:10087000F9CFC6D0E9DE94FD08C070FD02C09460D7
:100880000BC032DF94FFF9CF07C070FD02C0946047
:1008900003C02ADF94FDF9CFBAD0032D013F09F43C
:1008A00065CFEE2021F462CFEE2009F45FCF0091F6
:1008B0000601002321F400910501003250F000915F
:1008C000210192FD00270395009321019B7F0C33AA
:1008D00038F00FEFF02E80DE87DE9F7D7B7F02C039
:1008E000B3DE5FCF4DD070FF2FC0806490DE52D05A
:1008F00073DE78DE3BD070FF27C0806188DE51D088
:100900006BDE70DE3DD070FF1FC0806280DE5DD088
:1009100063DE68DE2BD070FF17C0906478DE5CD099
:100920005BDE60DE2DD070FF0FC071DE69D054DE5B
:1009300059DE1CD070FF08C06ADE69D04DDE52DE81
:1009400000910601002319F09062977F11CF977FE5
:10095000FF2041F0FA9429F00F2D013011F0023000
:1009600009F49860BFCFF894ACDE6ACB70FF0895AD
:1009700000B705FFFBCFB4DE00B705FFF7CF089542
:1009800070FF089500B705FDFBCFAADE00B705FD97
:10099000F7CF0895459A80FF439807EE00937C00B7
:1009A000089500E000936E0000007F7E7F7D81FD52
:1009B00002C076FD03C05B9880FF449A01E000937B
:1009C0006E0006EE00937C000895439A80FF5C98C9
:1009D00000EE00937C00089500E000936E0000009C
:1009E00070617F7D81FD02C076FD03C0449880FF69
:1009F000419A01E000936E0007EE00937C00089599
:100A00005C9A80FF459806EE00937C00089500E014
:100A100000936E0000007F7E706281FD02C076FD53
:100A200003C0419880FF5B9A01E000936E0000EEE6
:060A300000937C00089514
:00000001FF
